Link Map...

...Options...
EXE
ALIGNAddr:0x00001000		Alignfile:0x00000200		BASe:0x00400000
CODE:RX		DATA:RW		NODEBug		Defaultlibs
NODLLInitinstance		NODLLTerminstance		EXEPACK:2
EXPORTAll	NOExtdictionary	FIxed		NOFOrce
HEAP:0x00100000,0x00001000	NOIgnorecase	NOLInenumbers
MAP:C:\Programs\IBM\SOM\samples\somk\c\animals\animals.map	NOPAdding
PMTYPE:VIO	ROBAse:0x00000000		STACK:0x00100000,0x00001000
STUb		SUBSYSTEM:CONSOLE,04.00		VERSION:00.00	NAMElength:64000

...Segments...

 Start		Length	Name		Class

 00401000		BSS32		BSS
	at offset 00000000 bytes 000C8H from  "animals.obj" for "animals.obj(-1)|C:\Programs\IBM\SOM\samples\somk\c\animals\animals.c (BSS32:BSS)"
	at offset 000000C8 bytes 00004H from  "animals.obj" for "___somC_Animals_Animal_parentMtabs"
	at offset 000000CC bytes 00004H from  "animals.obj" for "___somC_Animals_M_Animal_parentMtabs"
	at offset 000000D0 bytes 00004H from  "animals.obj" for "___somC_Animals_Dog_parentMtabs"
	at offset 000000D4 bytes 00004H from  "animals.obj" for "___somC_Animals_Kennel_parentMtabs"
	at offset 000000D8 bytes 00004H from  "animals.obj" for "___somC_Animals_BigDog_parentMtabs"
	at offset 000000DC bytes 00004H from  "animals.obj" for "___somC_Animals_LittleDog_parentMtabs"

 00402000		CODE32		CODE
	at offset 00000000 bytes 00DA9H from  "animals.obj" for "animals.obj(-1)|C:\Programs\IBM\SOM\samples\somk\c\animals\animals.c (CODE32:CODE)"
	at offset 00000DB0 bytes 0020EH from  "main.obj" for "main.obj(-1)|C:\Programs\IBM\SOM\samples\somk\c\animals\main.c (CODE32:CODE)"
	at offset 00000DB0 bytes 00000H from  "main.obj" for "?main"
	at offset 00000FC0 bytes 0007AH from  "CPPRNO40.LIB(..\common\dde4strt.c)" for "?_start"
	at offset 00001040 bytes 00006H from  "CPPRNO40.LIB(..\common\crtweak1.c)" for "?_crtweak1"
	at offset 00001050 bytes 00001H from  "CPPRNO40.LIB(..\common\crtweak.c)" for "?_crtweak"
	at offset 00001051 bytes 001B7H from  "CPPRNO40.LIB(..\common\ix86\setuparg.asm)" for "CPPRNO40.LIB(23)|..\common\ix86\setuparg.asm (CODE32:CODE)"
	at offset 00001051 bytes 00000H from  "CPPRNO40.LIB(..\common\ix86\setuparg.asm)" for "?_setuparg"
	at offset 00001210 bytes 00044H from  "CPPRNO40.LIB(..\common\exit.c)" for "?exit"

 00403260		SEG0002		CODE
	at offset 00001260 bytes 003B3H from  "animals.obj" for "animals.obj(-1)|C:\Programs\IBM\SOM\samples\somk\c\animals\animals.c (SEG0002:CODE)"
	at offset 00001260 bytes 00000H from  "animals.obj" for "_Animals_LittleDogNewClass@8"
	at offset 000012E2 bytes 00000H from  "animals.obj" for "_Animals_BigDogNewClass@8"
	at offset 00001380 bytes 00000H from  "animals.obj" for "_Animals_KennelNewClass@8"
	at offset 000013E6 bytes 00000H from  "animals.obj" for "_Animals_DogNewClass@8"
	at offset 000014F4 bytes 00000H from  "animals.obj" for "_Animals_M_AnimalNewClass@8"
	at offset 00001556 bytes 00000H from  "animals.obj" for "_Animals_AnimalNewClass@8"
	at offset 00001614 bytes 00006H for "jump to _somPrintf"
	at offset 0000161A bytes 00006H for "jump to _somGetGlobalEnvironment@0"
	at offset 00001620 bytes 00006H for "jump to _somPCallResolve@12"
	at offset 00001626 bytes 00006H for "jump to _somBuildClass2@12"
	at offset 0000162C bytes 00006H for "jump to _somParentNumResolve@12"
	at offset 00001634 bytes 00004H for "pointer to _Animals_AnimalNewClass@8"
	at offset 00001638 bytes 00004H for "pointer to _Animals_DogNewClass@8"
	at offset 0000163C bytes 00004H for "pointer to _Animals_LittleDogNewClass@8"
	at offset 00001640 bytes 00004H for "pointer to _Animals_BigDogNewClass@8"
	at offset 00001644 bytes 00004H for "pointer to _Animals_AnimalClassData"
	at offset 00001648 bytes 00004H for "pointer to _Animals_M_AnimalClassData"
	at offset 0000164C bytes 00004H for "pointer to _Animals_KennelClassData"
	at offset 00001650 bytes 00004H for "pointer to _Animals_DogClassData"
	at offset 00001654 bytes 00004H for "pointer to _Animals_LittleDogClassData"
	at offset 00001658 bytes 00004H for "pointer to _Animals_BigDogClassData"
	at offset 0000165C bytes 00006H for "jump to ?malloc"
	at offset 00001662 bytes 00006H for "jump to ?_terminate"

 00404000		CONST32_RO		CONST
	at offset 00000000 bytes 00378H from  "animals.obj" for "animals.obj(-1)|C:\Programs\IBM\SOM\samples\somk\c\animals\animals.c (CONST32_RO:CONST)"
	at offset 00000378 bytes 00180H from  "main.obj" for "main.obj(-1)|C:\Programs\IBM\SOM\samples\somk\c\animals\main.c (CONST32_RO:CONST)"

 00405000		DATA32		DATA
	at offset 00000000 bytes 01060H from  "animals.obj" for "animals.obj(-1)|C:\Programs\IBM\SOM\samples\somk\c\animals\animals.c (DATA32:DATA)"
	at offset 00000004 bytes 00000H from  "animals.obj" for "_Animals_AnimalClassData"
	at offset 00000028 bytes 00000H from  "animals.obj" for "_Animals_AnimalCClassData"
	at offset 00000208 bytes 00000H from  "animals.obj" for "___somC_Animals_Animal_newNDMethodsArray"
	at offset 000003A0 bytes 00000H from  "animals.obj" for "_Animals_Animal_ClassInitBlock"
	at offset 000004A0 bytes 00000H from  "animals.obj" for "___somC_Animals_Animal_ClassInfo"
	at offset 000004A8 bytes 00000H from  "animals.obj" for "_Animals_M_AnimalClassData"
	at offset 000004C0 bytes 00000H from  "animals.obj" for "_Animals_M_AnimalCClassData"
	at offset 00000608 bytes 00000H from  "animals.obj" for "___somC_Animals_M_Animal_newNDMethodsArray"
	at offset 00000718 bytes 00000H from  "animals.obj" for "_Animals_M_Animal_ClassInitBlock"
	at offset 00000818 bytes 00000H from  "animals.obj" for "___somC_Animals_M_Animal_ClassInfo"
	at offset 00000820 bytes 00000H from  "animals.obj" for "_Animals_DogClassData"
	at offset 00000834 bytes 00000H from  "animals.obj" for "_Animals_DogCClassData"
	at offset 0000098C bytes 00000H from  "animals.obj" for "___somC_Animals_Dog_newNDMethodsArray"
	at offset 00000AA4 bytes 00000H from  "animals.obj" for "_Animals_Dog_ClassInitBlock"
	at offset 00000BA4 bytes 00000H from  "animals.obj" for "___somC_Animals_Dog_ClassInfo"
	at offset 00000BAC bytes 00000H from  "animals.obj" for "_Animals_KennelClassData"
	at offset 00000BB4 bytes 00000H from  "animals.obj" for "_Animals_KennelCClassData"
	at offset 00000C1C bytes 00000H from  "animals.obj" for "___somC_Animals_Kennel_newNDMethodsArray"
	at offset 00000C6C bytes 00000H from  "animals.obj" for "_Animals_Kennel_ClassInitBlock"
	at offset 00000D6C bytes 00000H from  "animals.obj" for "___somC_Animals_Kennel_ClassInfo"
	at offset 00000D74 bytes 00000H from  "animals.obj" for "_Animals_BigDogClassData"
	at offset 00000D78 bytes 00000H from  "animals.obj" for "_Animals_BigDogCClassData"
	at offset 00000DE0 bytes 00000H from  "animals.obj" for "_Animals_BigDog_ClassInitBlock"
	at offset 00000EE0 bytes 00000H from  "animals.obj" for "___somC_Animals_BigDog_ClassInfo"
	at offset 00000EE8 bytes 00000H from  "animals.obj" for "_Animals_LittleDogClassData"
	at offset 00000EEC bytes 00000H from  "animals.obj" for "_Animals_LittleDogCClassData"
	at offset 00000F58 bytes 00000H from  "animals.obj" for "_Animals_LittleDog_ClassInitBlock"
	at offset 00001058 bytes 00000H from  "animals.obj" for "___somC_Animals_LittleDog_ClassInfo"
	at offset 00001060 bytes 00004H from  "main.obj" for "main.obj(-1)|C:\Programs\IBM\SOM\samples\somk\c\animals\main.c (DATA32:DATA)"
	at offset 00001064 bytes 00004H from  "CPPRNO40.LIB(..\common\exit.c)" for "CPPRNO40.LIB(32)|..\common\exit.c (DATA32:DATA)"
	at offset 00001064 bytes 00000H from  "CPPRNO40.LIB(..\common\exit.c)" for "__exitflag"

 00406068		DDE4_DATA32		DATA
	at offset 00001068 bytes 00004H from  "CPPRNO40.LIB(..\common\ix86\exeentry.asm)" for "CPPRNO40.LIB(29)|..\common\ix86\exeentry.asm (DDE4_DATA32:DATA)"
	at offset 00001068 bytes 00000H from  "CPPRNO40.LIB(..\common\ix86\exeentry.asm)" for "__exeentry"
	at offset 0000106C bytes 00018H from  "CPPRNO40.LIB(..\common\ix86\setuparg.asm)" for "CPPRNO40.LIB(23)|..\common\ix86\setuparg.asm (DDE4_DATA32:DATA)"
	at offset 0000107C bytes 00000H from  "CPPRNO40.LIB(..\common\ix86\setuparg.asm)" for "__argc"
	at offset 00001080 bytes 00000H from  "CPPRNO40.LIB(..\common\ix86\setuparg.asm)" for "__argv"

...Constructor/Destructor pairs to run...
Init		Signature	Term	Signature

 Address		Imports by name
 00000000	Imp	"SOM_TraceLevel"	"som.dll"
 00000000	Imp	"SOM_TraceLevel"	"som.dll"
 00000000	Imp	"SOM_TraceLevel"	"som.dll"
 00000000	Imp	"SOM_TraceLevel"	"som.dll"
 00000000	Imp	"SOM_TraceLevel"	"som.dll"
 00000000	Imp	"_upool"	"cpprni40.dll"
 00000000	Imp	"SOM_TraceLevel"	"som.dll"
 00000000	Imp	"SOMObjectNewClass"	"som.dll"
 00000000	Imp	"somParentNumResolve"	"som.dll"
 00000000	Imp	"SOMClassClassData"	"som.dll"
 00000000	Imp	"malloc"	"cpprni40.dll"
 00000000	Imp	"SOMMalloc"	"som.dll"
 00000000	Imp	"SOMMalloc"	"som.dll"
 00000000	Imp	"SOM_TraceLevel"	"som.dll"
 00000000	Imp	"SOMClassClassData"	"som.dll"
 00000000	Imp	"SOMClassClassData"	"som.dll"
 00000000	Imp	"SOM_TraceLevel"	"som.dll"
 00000000	Imp	"SOMFree"	"som.dll"
 00000000	Imp	"SOM_TraceLevel"	"som.dll"
 00000000	Imp	"_fpreset"	"cpprni40.dll"
 00000000	Imp	"SOM_TraceLevel"	"som.dll"
 00000000	Imp	"GetCommandLineA"	"KERNEL32.dll"
 00000000	Imp	"SOMClassClassData"	"som.dll"
 00000000	Imp	"SOM_TraceLevel"	"som.dll"
 00000000	Imp	"SOMClassClassData"	"som.dll"
 00000000	Imp	"_terminate"	"cpprni40.dll"
 00000000	Imp	"SOMObjectClassData"	"som.dll"
 00000000	Imp	"SOM_TraceLevel"	"som.dll"
 00000000	Imp	"SOM_TraceLevel"	"som.dll"
 00000000	Imp	"SOM_TraceLevel"	"som.dll"
 00000000	Imp	"SOMObjectClassData"	"som.dll"
 00000000	Imp	"SOMClassClassData"	"som.dll"
 00000000	Imp	"SOMMalloc"	"som.dll"
 00000000	Imp	"SOM_TraceLevel"	"som.dll"
 00000000	Imp	"SOM_TraceLevel"	"som.dll"
 00000000	Imp	"SOMObjectClassData"	"som.dll"
 00000000	Imp	"SOMFree"	"som.dll"
 00000000	Imp	"SOM_TraceLevel"	"som.dll"
 00000000	Imp	"SOMFree"	"som.dll"
 00000000	Imp	"SOMFree"	"som.dll"
 00000000	Imp	"SOM_TraceLevel"	"som.dll"
 00000000	Imp	"_terminate"	"cpprni40.dll"
 00000000	Imp	"SOMObjectClassData"	"som.dll"
 00000000	Imp	"SOMMalloc"	"som.dll"
 00000000	Imp	"SOMMalloc"	"som.dll"
 00000000	Imp	"_runtime_heap"	"cpprni40.dll"
 00000000	Imp	"SOMObjectClassData"	"som.dll"
 00000000	Imp	"SOM_TraceLevel"	"som.dll"
 00000000	Imp	"SOMClassClassData"	"som.dll"
 00000000	Imp	"SOMFree"	"som.dll"
 00000000	Imp	"SOM_TraceLevel"	"som.dll"
 00000000	Imp	"SOM_TraceLevel"	"som.dll"
 00000000	Imp	"SOMClassClassData"	"som.dll"
 00000000	Imp	"somPrintf"	"som.dll"
 00000000	Imp	"SOM_TraceLevel"	"som.dll"
 00000000	Imp	"SOMClassClassData"	"som.dll"
 00000000	Imp	"SOMFree"	"som.dll"
 00000000	Imp	"SOM_TraceLevel"	"som.dll"
 00000000	Imp	"SOMClassClassData"	"som.dll"
 00000000	Imp	"SOMClassClassData"	"som.dll"
 00000000	Imp	"somGetGlobalEnvironment"	"som.dll"
 00000000	Imp	"SOMClassNewClass"	"som.dll"
 00000000	Imp	"SOMObjectClassData"	"som.dll"
 00000000	Imp	"_terminate"	"cpprni40.dll"
 00000000	Imp	"SOM_TraceLevel"	"som.dll"
 00000000	Imp	"SOM_TraceLevel"	"som.dll"
 00000000	Imp	"SOMRealloc"	"som.dll"
 00000000	Imp	"SOMClassNewClass"	"som.dll"
 00000000	Imp	"SOMFree"	"som.dll"
 00000000	Imp	"SOMClassClassData"	"som.dll"
 00000000	Imp	"somPCallResolve"	"som.dll"
 00000000	Imp	"SOMFree"	"som.dll"
 00000000	Imp	"SOMObjectClassData"	"som.dll"
 00000000	Imp	"SOM_TraceLevel"	"som.dll"
 00000000	Imp	"SOM_TraceLevel"	"som.dll"
 00000000	Imp	"SOMObjectClassData"	"som.dll"
 00000000	Imp	"SOM_TraceLevel"	"som.dll"
 00000000	Imp	"somBuildClass2"	"som.dll"

 Address		Publics by name
 00403050	"?_crtweak"
 00403040	"?_crtweak1"
 00403051	"?_setuparg"
 00402FC0	"?_start"
 00403210	"?exit"
 00402DB0	"?main"
 00403051	"CPPRNO40.LIB(23)|..\common\ix86\setuparg.asm (CODE32:CODE)"
 0040606C	"CPPRNO40.LIB(23)|..\common\ix86\setuparg.asm (DDE4_DATA32:DATA)"
 00406068	"CPPRNO40.LIB(29)|..\common\ix86\exeentry.asm (DDE4_DATA32:DATA)"
 00406064	"CPPRNO40.LIB(32)|..\common\exit.c (DATA32:DATA)"
 00405028	"_Animals_AnimalCClassData"
 00405004	"_Animals_AnimalClassData"
 00403556	"_Animals_AnimalNewClass@8"
 004053A0	"_Animals_Animal_ClassInitBlock"
 00405D78	"_Animals_BigDogCClassData"
 00405D74	"_Animals_BigDogClassData"
 004032E2	"_Animals_BigDogNewClass@8"
 00405DE0	"_Animals_BigDog_ClassInitBlock"
 00405834	"_Animals_DogCClassData"
 00405820	"_Animals_DogClassData"
 004033E6	"_Animals_DogNewClass@8"
 00405AA4	"_Animals_Dog_ClassInitBlock"
 00405BB4	"_Animals_KennelCClassData"
 00405BAC	"_Animals_KennelClassData"
 00403380	"_Animals_KennelNewClass@8"
 00405C6C	"_Animals_Kennel_ClassInitBlock"
 00405EEC	"_Animals_LittleDogCClassData"
 00405EE8	"_Animals_LittleDogClassData"
 00403260	"_Animals_LittleDogNewClass@8"
 00405F58	"_Animals_LittleDog_ClassInitBlock"
 004054C0	"_Animals_M_AnimalCClassData"
 004054A8	"_Animals_M_AnimalClassData"
 004034F4	"_Animals_M_AnimalNewClass@8"
 00405718	"_Animals_M_Animal_ClassInitBlock"
 004054A0	"___somC_Animals_Animal_ClassInfo"
 00405208	"___somC_Animals_Animal_newNDMethodsArray"
 004010C8	"___somC_Animals_Animal_parentMtabs"
 00405EE0	"___somC_Animals_BigDog_ClassInfo"
 004010D8	"___somC_Animals_BigDog_parentMtabs"
 00405BA4	"___somC_Animals_Dog_ClassInfo"
 0040598C	"___somC_Animals_Dog_newNDMethodsArray"
 004010D0	"___somC_Animals_Dog_parentMtabs"
 00405D6C	"___somC_Animals_Kennel_ClassInfo"
 00405C1C	"___somC_Animals_Kennel_newNDMethodsArray"
 004010D4	"___somC_Animals_Kennel_parentMtabs"
 00406058	"___somC_Animals_LittleDog_ClassInfo"
 004010DC	"___somC_Animals_LittleDog_parentMtabs"
 00405818	"___somC_Animals_M_Animal_ClassInfo"
 00405608	"___somC_Animals_M_Animal_newNDMethodsArray"
 004010CC	"___somC_Animals_M_Animal_parentMtabs"
 0040607C	"__argc"
 00406080	"__argv"
 00406068	"__exeentry"
 00406064	"__exitflag"
 00401000	"animals.obj(-1)|C:\Programs\IBM\SOM\samples\somk\c\animals\animals.c (BSS32:BSS)"
 00402000	"animals.obj(-1)|C:\Programs\IBM\SOM\samples\somk\c\animals\animals.c (CODE32:CODE)"
 00404000	"animals.obj(-1)|C:\Programs\IBM\SOM\samples\somk\c\animals\animals.c (CONST32_RO:CONST)"
 00405000	"animals.obj(-1)|C:\Programs\IBM\SOM\samples\somk\c\animals\animals.c (DATA32:DATA)"
 00403260	"animals.obj(-1)|C:\Programs\IBM\SOM\samples\somk\c\animals\animals.c (SEG0002:CODE)"
 00403662	"jump to ?_terminate"
 0040365C	"jump to ?malloc"
 00403626	"jump to _somBuildClass2@12"
 0040361A	"jump to _somGetGlobalEnvironment@0"
 00403620	"jump to _somPCallResolve@12"
 0040362C	"jump to _somParentNumResolve@12"
 00403614	"jump to _somPrintf"
 00402DB0	"main.obj(-1)|C:\Programs\IBM\SOM\samples\somk\c\animals\main.c (CODE32:CODE)"
 00404378	"main.obj(-1)|C:\Programs\IBM\SOM\samples\somk\c\animals\main.c (CONST32_RO:CONST)"
 00406060	"main.obj(-1)|C:\Programs\IBM\SOM\samples\somk\c\animals\main.c (DATA32:DATA)"
 00403644	"pointer to _Animals_AnimalClassData"
 00403634	"pointer to _Animals_AnimalNewClass@8"
 00403658	"pointer to _Animals_BigDogClassData"
 00403640	"pointer to _Animals_BigDogNewClass@8"
 00403650	"pointer to _Animals_DogClassData"
 00403638	"pointer to _Animals_DogNewClass@8"
 0040364C	"pointer to _Animals_KennelClassData"
 00403654	"pointer to _Animals_LittleDogClassData"
 0040363C	"pointer to _Animals_LittleDogNewClass@8"
 00403648	"pointer to _Animals_M_AnimalClassData"

 Address		Publics by value
 00401000	"animals.obj(-1)|C:\Programs\IBM\SOM\samples\somk\c\animals\animals.c (BSS32:BSS)"
 004010C8	"___somC_Animals_Animal_parentMtabs"
 004010CC	"___somC_Animals_M_Animal_parentMtabs"
 004010D0	"___somC_Animals_Dog_parentMtabs"
 004010D4	"___somC_Animals_Kennel_parentMtabs"
 004010D8	"___somC_Animals_BigDog_parentMtabs"
 004010DC	"___somC_Animals_LittleDog_parentMtabs"
 00402000	"animals.obj(-1)|C:\Programs\IBM\SOM\samples\somk\c\animals\animals.c (CODE32:CODE)"
 00402DB0	"main.obj(-1)|C:\Programs\IBM\SOM\samples\somk\c\animals\main.c (CODE32:CODE)"
 00402DB0	"?main"
 00402FC0	"?_start"
 00403040	"?_crtweak1"
 00403050	"?_crtweak"
 00403051	"CPPRNO40.LIB(23)|..\common\ix86\setuparg.asm (CODE32:CODE)"
 00403051	"?_setuparg"
 00403210	"?exit"
 00403260	"animals.obj(-1)|C:\Programs\IBM\SOM\samples\somk\c\animals\animals.c (SEG0002:CODE)"
 00403260	"_Animals_LittleDogNewClass@8"
 004032E2	"_Animals_BigDogNewClass@8"
 00403380	"_Animals_KennelNewClass@8"
 004033E6	"_Animals_DogNewClass@8"
 004034F4	"_Animals_M_AnimalNewClass@8"
 00403556	"_Animals_AnimalNewClass@8"
 00403614	"jump to _somPrintf"
 0040361A	"jump to _somGetGlobalEnvironment@0"
 00403620	"jump to _somPCallResolve@12"
 00403626	"jump to _somBuildClass2@12"
 0040362C	"jump to _somParentNumResolve@12"
 00403634	"pointer to _Animals_AnimalNewClass@8"
 00403638	"pointer to _Animals_DogNewClass@8"
 0040363C	"pointer to _Animals_LittleDogNewClass@8"
 00403640	"pointer to _Animals_BigDogNewClass@8"
 00403644	"pointer to _Animals_AnimalClassData"
 00403648	"pointer to _Animals_M_AnimalClassData"
 0040364C	"pointer to _Animals_KennelClassData"
 00403650	"pointer to _Animals_DogClassData"
 00403654	"pointer to _Animals_LittleDogClassData"
 00403658	"pointer to _Animals_BigDogClassData"
 0040365C	"jump to ?malloc"
 00403662	"jump to ?_terminate"
 00404000	"animals.obj(-1)|C:\Programs\IBM\SOM\samples\somk\c\animals\animals.c (CONST32_RO:CONST)"
 00404378	"main.obj(-1)|C:\Programs\IBM\SOM\samples\somk\c\animals\main.c (CONST32_RO:CONST)"
 00405000	"animals.obj(-1)|C:\Programs\IBM\SOM\samples\somk\c\animals\animals.c (DATA32:DATA)"
 00405004	"_Animals_AnimalClassData"
 00405028	"_Animals_AnimalCClassData"
 00405208	"___somC_Animals_Animal_newNDMethodsArray"
 004053A0	"_Animals_Animal_ClassInitBlock"
 004054A0	"___somC_Animals_Animal_ClassInfo"
 004054A8	"_Animals_M_AnimalClassData"
 004054C0	"_Animals_M_AnimalCClassData"
 00405608	"___somC_Animals_M_Animal_newNDMethodsArray"
 00405718	"_Animals_M_Animal_ClassInitBlock"
 00405818	"___somC_Animals_M_Animal_ClassInfo"
 00405820	"_Animals_DogClassData"
 00405834	"_Animals_DogCClassData"
 0040598C	"___somC_Animals_Dog_newNDMethodsArray"
 00405AA4	"_Animals_Dog_ClassInitBlock"
 00405BA4	"___somC_Animals_Dog_ClassInfo"
 00405BAC	"_Animals_KennelClassData"
 00405BB4	"_Animals_KennelCClassData"
 00405C1C	"___somC_Animals_Kennel_newNDMethodsArray"
 00405C6C	"_Animals_Kennel_ClassInitBlock"
 00405D6C	"___somC_Animals_Kennel_ClassInfo"
 00405D74	"_Animals_BigDogClassData"
 00405D78	"_Animals_BigDogCClassData"
 00405DE0	"_Animals_BigDog_ClassInitBlock"
 00405EE0	"___somC_Animals_BigDog_ClassInfo"
 00405EE8	"_Animals_LittleDogClassData"
 00405EEC	"_Animals_LittleDogCClassData"
 00405F58	"_Animals_LittleDog_ClassInitBlock"
 00406058	"___somC_Animals_LittleDog_ClassInfo"
 00406060	"main.obj(-1)|C:\Programs\IBM\SOM\samples\somk\c\animals\main.c (DATA32:DATA)"
 00406064	"CPPRNO40.LIB(32)|..\common\exit.c (DATA32:DATA)"
 00406064	"__exitflag"
 00406068	"CPPRNO40.LIB(29)|..\common\ix86\exeentry.asm (DDE4_DATA32:DATA)"
 00406068	"__exeentry"
 0040606C	"CPPRNO40.LIB(23)|..\common\ix86\setuparg.asm (DDE4_DATA32:DATA)"
 0040607C	"__argc"
 00406080	"__argv"

...Import library list...
Library	UsageCount
"som.dll"	13
"cpprni40.dll"	5
"KERNEL32.dll"	1

Program entry point at 00402FC0	"?_start"

